:100000009729A501A400B3172730A30010301420AE
:100010000330A300E8301420A30164301420A301AE
:100020000A30142024081F28A2002508A100240853
:10003000A00055212008031DB313B31B0800303E58
:1000400022280408A2008316051183120930A30098
:1000500003103520A20CA30B2928031435200330EC
:10006000A100E8302F210314922903183A28000038
:1000700005113C2805153C280030A10062302F29CD
:10008000A501A400B3172730A3001030532003307C
:10009000A300E8305320A30164305320A3010A30A9
:1000A000532024085E28A2002508A1002408A000EF
:1000B00055212008031DB313B31B0800303EA600D2
:1000C000360884000930A70003106B20A60CA70B8C
:1000D000652803146B288413B31D7A2800083404A0
:1000E000331D34068000841700083404031C3406D2
:1000F0008000852800083404031C340633193406B4
:100100008000841734098005852800308A00330D6B
:100110000639A0009220A10000308A00200A922017
:1001200000002F29963E03188A0A82000134893480
:1001300003342934003450340C34ED342C08A0003E
:100140002D08A1000130A200A3016400CE20031CF1
:10015000B928A20BA528FF30A3070318A528A007DC
:10016000031CA107031C08006430A2000030A30098
:10017000A528E920A801A2010930A300EA20CE2089
:100180000318A80AAB1EA801A20CA30BBE28AB1A29
:10019000A213A20DEA2003142208080036088400E6
:1001A000340884178004841300052B1B3406FF3E9B
:1001B0000800A40029080314031992298D21031CA7
:1001C0000800A0002408840020088000A40AA903D5
:1001D000DA2833172B081F39003EA1002A08043EF5
:1001E0000318A10A331F2F293313A0000310A10CF9
:1001F000A00C0310A10C200C2F29B31329080319FC
:10020000B3170430A800250E0A2125080A21240E60
:100210000A2124080F39F63E0318073E0A3E10292A
:10022000A000A8030319B313290803191A292802E7
:10023000031808002008031DB313B31B0800303E49
:100240008D29A301A200FF30A207031CA307031CF2
:1002500092290330A100E3302F212329A101F43E8C
:10026000A000A109FE30031C3829A0070318352976
:10027000A0076400A10F3529000020183F2920188D
:1002800041290800A000A11B872120089229A20073
:100290002008A6002408A0002608A4002108A60023
:1002A0002508A1002608A5005729A501A4011030A2
:1002B000A600210DA40DA50D2208A4022308031CED
:1002C000230FA50203186B292208A407230803188B
:1002D000230FA5070310A00DA10DA60B5929200877
:1002E00092291030A800A101A001A70CA60C031CA4
:1002F0007F292208A00723080318230FA107A10CB8
:10030000A00CA50CA40CA80B752924089229A009FF
:10031000A109A00A0319A10A0800840031088A0073
:1003200030088200831303138312640008008830AE
:100330008B00831675308F00831207309900831667
:10034000133085009F0183129F0183167F30810047
:100350000330950083120530B6002030B40006301B
:10036000B3000D305F200B30A300B83022217C3069
:1003700022209D302220FE30222080302220423058
:100380002220433022204D302220203022204730AE
:1003900022206130222075302220673022206530F3
:1003A00022202030222020302220563022203230BD
:1003B00022202E3022203030222035302220FE30E4
:1003C0002220C03022207730222077302220773040
:1003D00022202E3022203130222035302220303091
:1003E00022206D30222070302220673022202E30D3
:1003F0002220633022206F3022202E3022207530C0
:1004000022206B3022200730A300D0302221FE3082
:100410002220013022200530B6002030B400063002
:10042000B30043305F204C305F2045305F204130C7
:100430005F2052305F2044305F2041305F205430D5
:100440005F2041305F200D305F204D305F20533002
:100450005F2047305F202C305F2020305F2042300B
:100460005F2043305F204D305F2020305F204730D9
:100470005F2061305F2075305F2067305F2065301E
:100480005F2020305F2044305F2061305F20743077
:100490005F2061305F200D305F200530B6001030E6
:1004A000B4005430AA002030AB00FA30AC00AD01EB
:1004B0009E20031C4B2D873C031D582A0B30A9009E
:1004C0009E30B000B1013830D920031C4B2D87304D
:1004D000D900DA0164000A305A020318782A5A084F
:1004E000383E84000008D2005208D907DA0F6A2A81
:1004F000D909D90A7F30D905640042085902031D81
:100500004D2A0530B6001030B4005430AA00203017
:10051000AB00FA30AC00AD019E20031C4B2DAA3C71
:10052000031D8C2A0B30A9009E30B000B10143306E
:10053000D920031C4B2DAA30D900DA0164000A30FF
:100540005A020318AC2A5A08433E84000008D2001D
:100550005208D907DA0F9E2AD909D90A7F30D9055E
:1005600064004D085902031D812A64008518FE2A83
:100570000530A300DC302221FE3022200130222071
:10058000FE302220803022200130DA006400093061
:100590005A020318DB2A0230A9005A08383E8400A8
:1005A0000008D2005208A400A5012130B000B1011A
:1005B000FD20DA0FC62AFE302220C0302220013072
:1005C000DA00640009305A020318F62A0230A90042
:1005D0005A08433E84000008D2005208A400A50136
:1005E0002130B000B101FD20DA0FE12A0530A3006F
:1005F000DC302221FE302220013022203908A600E2
:10060000A7010230A200A3017121DE0007303A05E4
:10061000DA005A08A600A7018030A200A3017121C8
:10062000D2002508D3003B085207D0005308031816
:10063000013ED100FE302220803022205E080120C1
:10064000203022205008A0005108A1000A30A2004A
:10065000A3015521D2002108D3005308A500520858
:1006600002202E3022205008A0005108A1000A309C
:10067000A200A30155212408D2002508D300530865
:10068000A5005208022025302220203022203C08DC
:10069000A600A7018030A200A3017121D200250885
:1006A000D3003D08D2070318D30A00305202CE000F
:1006B0000830031C013E5302CF00CF1B5B14CF1F39
:1006C0005B104F08A1004E084221CE002108CF0048
:1006D0004E08A6004F08A700C430A2000930A300AE
:1006E0007121CE002508CF000230A3000030472141
:1006F000CE002108CF0064005B1C812B2D30D80078
:10070000832B2B30D8004E08A0004F08A100643086
:10071000A200A30155212408D2002508D3005208C5
:10072000A0005308A1000A30A200A3015521DA005D
:100730004E08A0004F08A1006430A200A30155217B
:10074000CE002108CF00580822204F08A5004E08EF
:1007500002202E3022205A08012020302220203072
:100760002220640020303F020318C02B3F08203CA9
:10077000D4000030031CFF3ED5002D30DC00C92B17
:10078000E0303F07D400FF300318013ED5002B3086
:10079000DC006400203040020318D82B4008203CC5
:1007A000D6000030031CFF3ED7002D30DD00E12BCA
:1007B000E0304007D600FF300318013ED7002B3051
:1007C000DD00640005186A2C64005C082D3C031DE4
:1007D0000A2C5408A6005508A7001230A200A30155
:1007E0007121D2002508D3005208A0005308A100AF
:1007F0000A30A200A3015521D2002108D3005208DB
:10080000203CD4005308031C013E003CD5002B3093
:10081000DC00272C5408A6005508A7001230A200BF
:10082000A3017121D2002508D3005208A00053086B
:10083000A1000A30A200A3015521D2002108D30053
:1008400020305207D40053080318013ED50064003D
:100850005D082D3C031D4D2C5608A6005708A70027
:100860001230A200A3017121D2002508D300520842
:10087000A0005308A1000A30A200A3015521D20014
:100880002108D3005208203CD6005308031C013E27
:10089000003CD7002B30DD006A2C5608A600570814
:1008A000A7001230A200A3017121D2002508D300B5
:1008B0005208A0005308A1000A30A200A30155214C
:1008C000D2002108D30020305207D6005308031865
:1008D000013ED700FE302220C03022205C082220BA
:1008E0005508A5005408022048302220203022203C
:1008F0005D0822205708A500560802204C3022200F
:1009000020302220533022200230A9004808A400C1
:10091000A5012130B000B101FD202030222020307F
:1009200022200530B6002030B4000630B300443039
:100930005F2041305F2054305F2041305F202C30F9
:100940005F2054305F2049305F204D305F204530BC
:100950005F202C305F205E0840202C305F2058083C
:100960005F202C305F204F08A5004E0841202C301E
:100970005F205108A500500841202C305F205C0802
:100980005F202C305F205508A500540841202C30F2
:100990005F205D085F202C305F205708A5005608B7
:1009A00041200D305F20640085184A2D0530B600C7
:1009B0002030B4000630B30044305F2041305F2067
:1009C00054305F2041305F202C305F2054305F2056
:1009D00049305F204D305F2045305F202C305F2054
:1009E000873040202C305F20DA0164000B305A023F
:1009F00003180B2D0530B6002030B4000630B300CC
:100A00005A08383E84000008D200520840202C309A
:100A10005F20DA0FF52C0530B6002030B400063028
:100A2000B3000D305F2044305F2041305F205430F0
:100A30005F2041305F202C305F2054305F204930F0
:100A40005F204D305F2045305F202C305F20AA3082
:100A500040202C305F20DA0164000B305A0203186A
:100A6000422D0530B6002030B4000630B3005A08DD
:100A7000433E84000008D200520840202C305F2002
:100A8000DA0F2C2D0530B6002030B4000630B3004C
:100A90000D305F204D2AFE30222001302220FE3012
:100AA0002220803022204E3022206F302220203021
:100AB000222042302220433022204D30222020307C
:100AC00022204430222061302220743022206130E4
:100AD0002220213022200330A300E83022214D2A99
:02400E009C3CD8
:00000001FF
